:0300000002000EED
:0300030002019F58
:20000B0002019675811FD2AFD2A91201A280FE12001B80FBC82581C822C92581C97A002224
:20002B00D083D082CF2581F581CFC082C08322CF2581F581CF22FBE493CB22FCE493FB7492
:20004B000193CC22FAE493F9740193CA2229F9E5F03AFA227C00CB30E7011CCB2275F0009B
:20006B0030E70215F022FDE493FF7401934F7004A3A3800C740293B50510740393B5F00A99
:20008B00E493C0E0740193C0E022A3A3A3A380D7FEEBA4FD8EF0ECA4FCEB8EF0A4C5F02C0F
:2000AB002DC5F02211B58EF0ED22C002C001AAF0F97E007D007F11C3E933F9EA33FADF0867
:2000CB00F5F0E9D001D00222ED33FDEE33FEC3ED9BF5F0EE9C40E0ADF0FED380DBBB0001E7
:2000EB0022C333C5F033C5F0DBF722BB000122C3C5F013C5F013DBF722240280022401C595
:20010B00F03400C5F022C394028003C39401C5F09400C5F0223116F4C5F0F4C5F02245F095
:20012B007022042231784024801A3178401E7014801A3178400E7014800A3178500E8004A0
:20014B00318C6008E4F5F022318C60F8E4F5F00422318C40F780ED318C40F170E780ED313C
:20016B008C40E170E780DD318C50E180D7C39BC5F09C20E70720D207C345F02220D2F9D340
:20018B0022C5F0C39C7003E5F09B22758CDC758A0005083205083274FFF512E4F5087412DE
:2001AB00F50DE4F50CE4F50A74FFF51DE4F50E7412F5197401F51A7412F51B7402F51CE4E5
:2001CB00F51FE4F5F079157A001200587440F7740175F00079157A001200587440F77402AD
:2001EB0075F00079157A001200587440F7740375F00079157A001200587440F7748075F020
:20020B0025C0E0C0F012079E15811581740175F00045F07003020256E5081200687B0112AA
:20022B00005F12012F700302023B1202C8020223E4F50812025712036F12042612072A12FC
:20024B0004781206961206C602021722E5090509E50975F0007B647C0012017270030202A8
:20026B00C7E4F509E50E4405F50E7432F511E50A050AE50A75F0007B3C7C00120172700362
:20028B000202C7E4F50AE50E4402F50EE50C050CE50C75F0007B3C7C0012017270030202E2
:2002AB00C7E4F50CE50D050DE50D75F0007B187C0012017270030202C7E4F50D22058105C7
:2002CB00817408F51474FFF51DE4F5F078FD12001FF608A6F078FD12001FE60886F07B04FC
:2002EB007C0012012F701902036A78FD12001FE60886F012010818F608A6F012011680D5EE
:20030B00E514F45512F5B078FD12001FE60886F079157A00120058E7F4F590740175F00023
:20032B00C0E0C0F01207551581158174FFF590E5B054101200687B0012005F12014B7003A0
:20034B0002035978FD12001FE60886F0F51DE51475F0007B017C001200F6F5140202F515A3
:20036B0081158122E4F5F079157A00120058E50C75F0007B0A7C001200AFC001C00279C129
:20038B007A0712005889828A83E493D007D000F6740175F00079157A00120058E50C75F099
:2003AB00007B0A7C001200B5C001C00279C17A0712005889828A83E493D007D000F6740220
:2003CB0075F00079157A00120058E50D75F0007B0A7C001200AFC001C00279C17A071200D2
:2003EB005889828A83E493D007D000F6740375F00079157A00120058E50D75F0007B0A7CC8
:20040B00001200B5C001C00279C17A0712005889828A83E493D007D000F622E50E54047554
:20042B00F0007B007C001201537003020477E5111511E51175F0007B007C0012015370032D
:20044B00020471740175F00079157A00120058E74480F7740275F00079157A00120058E7F8
:20046B004480F7020477E50E54FBF50E22E51D1200687BFF12005F12015370030204DEE5C9
:20048B000E548075F0007B007C0012014B70030204DEE50E4480F50E7432F51EE51D1200D7
:2004AB00689004CA0200711205BD0204DE1205140204DE1204F80204DE1204DF0204DEC4A2
:2004CB00040300BE040200B8040100B20400000000DE0422E50D050DE50D75F0007B187C65
:2004EB000012014B70030204F7E4F50D22E50C050CE4F50AE50C75F0007B3C7C0012014B4F
:20050B007003020513E4F50C22E51F051FE51F1200687B0112005F12014B7003020571E57B
:20052B000DF519E50CF51AE4F5F079157A00120058E4F7740175F00079157A0012005874BF
:20054B0068F7740275F00079157A001200587478F7740375F00079157A001200587471F7D7
:20056B00120650020577E4F51F12057822E50DF51BE50CF51CE4F5F079157A00120058742E
:20058B0063F7740175F00079157A001200587463F7740275F00079157A001200587478F7AC
:2005AB00740375F00079157A001200587471F7020650E512F4447FF512548075F0007B0045
:2005CB007C0012014B7003020613E4F5F079157A00120058E4F7740175F00079157A00129E
:2005EB000058E4F7740275F00079157A001200587468F7740375F00079157A0012005874DB
:20060B0078F712065002064FE4F5F079157A00120058E4F7740175F00079157A001200583F
:20062B007463F7740275F00079157A001200587463F7740375F00079157A0012005874788C
:20064B00F71206502205810581E4F5F078FD12001FF608A6F078FD12001FE60886F07BF486
:20066B007C0112012F701902069178FD12001FE60886F012010818F608A6F012011680D53F
:20068B001202C80206751581158122E50E548075F0007B007C0012015370030206C5E51EDC
:2006AB00151EE51E1200687B0012005F12014B70030206C5E50E547FF50E22E50E5401754D
:2006CB00F0007B007C001201537003020729E50E54FEF50EE50D75F000AB197C0012014BE0
:2006EB00600CE50C75F000AB1A7C0012014B45F07003020704747FF512E50D75F000AB1BC2
:20070B007C0012014B600CE50C75F000AB1C7C0012014B45F0700302072974FFF5122274A7
:20072B000375F00079157A00120058E775F0007B3F7C0012014B7003020754740375F00048
:20074B0079157A00120058E4F72205810581E4F5F078FD12001FF608A6F078FD12001FE684
:20076B000886F078F912001F860308860412012F701902079978FD12001FE60886F01201A9
:20078B000818F608A6F012011680CF020780158115812278FB12001F860308860474807523
:2007AB00F0701200B5120120758921F58DF58B758859759852223F0C765E4D5B7B0E7F5FAE
:00000001FF
